:100000004AC17EC105C362C161C160C15FC15EC139
:100010005DC15CC15BC15AC159C158C157C1120110
:10002000100100000008C016D927000101020301D9
:1000300009022200010100800309040000010300FD
:100040000000092101010001227700070581030852
:1000500000640600FF0901A101850715002501754F
:100060000195041A20022A230289069909B10295F2
:100070000109FF790AB10209FE790BB1820A260251
:10008000790CB182B103850326FC3F6701000100B2
:10009000550E36135B470F9B0000751095017904D0
:1000A00009E7B1A28501790409E78122850526AC1B
:1000B0000D6501550C3500461027790509EAB1B2E6
:1000C0008501790509EA8122C0FD0002012F014C5A
:1000D000016601750186019C01AC01B301CE01D41A
:1000E00001E801FD000201F6014C01110221023379
:1000F00002460254025B02710277028702D087D067
:100100008900686166746D616E6E23736F667477C3
:1001100061726520287777772E74752D6368656D19
:100120006E69747A2E64652F7E6865686129005354
:10013000485431312054656D706572617475722F49
:100140004C7566746665756368746500686568619A
:100150004068727A2E74752D6368656D6E69747A65
:100160002E64653A01004C75667474656D70657235
:10017000617475720052656C6174697665204665BC
:10018000756368746500526564757A696572746533
:10019000204175666CC3B673756E67004B65696EFA
:1001A000204F54502D52656C6F6164004865697A28
:1001B000657200546573746D6F6475732C206E697D
:1001C0006368742062656E75747A656E2100466F8F
:1001D0006B757300C39C62657274726167756E673C
:1001E000736665686C657200556E746572737061D4
:1001F0006E6E756E670053485431312054656D70D2
:10020000657261747572652F48756D69646974797A
:10021000004169722054656D706572617475726514
:100220000052656C61746976652048756D69646912
:1002300074790052656475636564207265736F6CD0
:100240007574696F6E004E6F204F54502072656C4C
:100250006F61640048656174657200546573742051
:100260006D6F64652C20646F206E6F7420757365EC
:1002700000466F637573005472616E736665722019
:100280006661696C656400456E64204F662042615A
:1002900074746572790011241FBECFE5D2E0DEBF11
:1002A000CDBF10E0A0E6B0E0E8EAFCE002C00590B7
:1002B0000D92A436B107D9F710E0A4E6B0E001C072
:1002C0001D92AE39B107E1F70FD3ECC499CEA82F38
:1002D000B92F80E090E041E050EA60956F5F58F4FC
:1002E0002D9138EF82279795879510F084279527D1
:1002F0003F5FC8F3F3CF0895EADF8D939D93089590
:10030000CF93CFB7CF93C395B29BE9F7B29B0EC003
:10031000B29B0CC0B29B0AC0B29B08C0B29B06C085
:10032000B29B04C0C2B7C8BD8D9ACEC00F92DF93F6
:10033000C0918100DD27C857DF4F012EB29B03C05B
:10034000DF910F90E3CF2F930F931F934F932FEFD6
:100350004F6F06B302FB20F95F933F9350E03BE001
:1003600065C016B30126502952FDC89556B3012722
:1003700002FB25F92F7306B3B1F05027102712FBAB
:1003800026F906B22230F0F000C016B3012702FBB6
:1003900027F90126502906B22430E8F54F77206866
:1003A00016B30000F6CF50274F7D206206B2102F03
:1003B000000000C006B300265029102712FB26F9C2
:1003C00006B2E2CF4F7B06B3206400C0DACF01262D
:1003D0005029167006B269F14E7F2160012F16B3C5
:1003E00028C0002650294D7F06B22260102F29C058
:1003F000012650294B7F06B22460012F2DC016B371
:1004000001265029477F2860000006B22EC04F7E8B
:1004100006B3206130C0422706B349930026502915
:10042000102706B24FEF12FB20F9297F16B379F29D
:10043000167049F10126502906B2012702FB21F965
:10044000237F06B371F2002650293150D0F006B256
:10045000102712FB22F9277E16B351F201265029EC
:10046000012702FB06B223F92F7C49F2000006B3F4
:10047000102712FB24F90026502906B22F7939F2F1
:1004800070CF002717C03B503195C31BD040088167
:10049000033CF1F00B34E1F020917F001981110F42
:1004A0001213EFCF4A81441F093639F10D3211F092
:1004B000013E39F7009386003F915F914F911F9164
:1004C0000F912F91DF910F90CF91CFBFCF911895C2
:1004D00000918600002381F310918400112379F5A7
:1004E00034307AF1309384000093800010918100C1
:1004F0003BE0311B3093810024C000918400013027
:10050000F4F40AE54F7049F43091610034FD1AC0EB
:1005100000936100C9E6D0E019C03091620034FD5B
:1005200011C000936200C4E7D0E010C0052710E0BE
:1005300000C021C0052710E0C89508BB14C03AE5EB
:1005400001C032ED032EC0E0D0E032E017B31660F8
:10055000C29A08B317BB56E020E84FEF20FF0527EB
:1005600008BB279517951C3F28F700004552B0F7A8
:1005700020FF0527279508BB17951C3FB8F6299142
:100580003A9561F7097F10918500110F08BBC250A1
:10059000D04011F010937F00046017B3197F402FF3
:1005A000497F54E05A95F1F708BB17BB48BB84CF8D
:1005B0008DE08A95F1F7089587FF03C0BC98C49A2F
:1005C00002C0C498BC9A9DE09A95F1F7C39A9DE049
:1005D0009A95F1F7880FB4998160C3989DE09A9538
:1005E000F1F7615049F7089568E0E6DF80E861E0DF
:1005F000E3DF08950F931F93082F8FEF68E0DCDF90
:10060000182F802F61E0D8DF812F1F910F9108955F
:100610001895442079F020E0C39A8DE0982F9A95A0
:10062000F1F7982F9A95F1F7C3988A95F1F72F5F14
:10063000293091F7C39A8DE0982F9A95F1F7C498D5
:10064000BC9A982F9A95F1F7C398982F9A95F1F73D
:10065000982F9A95F1F7C39A982F9A95F1F7BC982D
:10066000C49A982F9A95F1F7C3988A95F1F708954F
:10067000382F932D20E0892F87958827879583270A
:10068000880F880B8C7896959827330F2F5F28302A
:1006900091F7392E0895CF93DF93FC018281282FA3
:1006A00030E02D30310510F090E076C08481220FCB
:1006B000331F873021F4F901E753FF4F03C0F901DD
:1006C000ED51FF4F45915491A0EAB0E051C04F5F0A
:1006D0005F4FE130F10539F588EF9FEF9FBB8EBB8F
:1006E000E09A8DB3282F30E0F09AE09A8DB3D82F9E
:1006F000C0E02C2B3D2BFD0164E0C901892F992717
:1007000082958F708A30910508F00796C096819384
:100710009193615011F418962BC074E0220F331F8F
:100720007A95E1F7EACFE7FF21C0CF0136E0880FE5
:10073000991F3A95E1F79F70FA014F5F5F4FE4917F
:10074000F0E0EF73F070E82BF92BF3FF0FC0CF014F
:1007500026E0880F991F2A95E1F7FA014F5F5F4F56
:10076000E491F0E0EF73F070E82BF92BED93FD933B
:10077000FA018491E82FF0E0309709F0A8CF2EE934
:1007800030E09A2F921B90939E0083E080939F000D
:100790003093830020938200892FDF91CF910895B9
:1007A00086B3867009F08895A8958D9B36C098B55C
:1007B0009E5080916400981B88B5809364008D984A
:1007C000993F1CF481B78F5F81BF98301CF081B7CF
:1007D000815081BF8091660090916700019690934F
:1007E000670080936600209168002223B1F0809119
:1007F0001E0190911F01019790931F0180931E018C
:10080000892B59F4822F90E0880F991F880F991F28
:1008100090931F0180931E018E9A08950F931F934A
:10082000CF93DF93082FF5DE802FDEDE882329F0BB
:1008300044244394CFEFDFEF3DC0322C802F18DFEC
:10084000C0916600D091670080E28ABF80E68BBFCE
:10085000B09A11C080916600909167008C1B9D0B2F
:100860008159914038F080E48BBF44244394CEEF0B
:10087000DFEF20C095DFB499EDCFB09A80E48BBF55
:1008800080E0B8DE182FC82FD0E0F2DE073021F468
:10089000BFE02B2E21220AC080E0ACDE182FE8DE5C
:1008A0009C2F8827C12FD0E0C82BD92B8FEFA2DE39
:1008B000432C481ACE01DF91CF911F910F910895DB
:1008C00083E0ACDF97FD0EC090932201809321015D
:1008D00085E0A4DF97FD06C0909324018093230157
:1008E00081E0089580E0089584B714BE479A98E1A6
:1008F00091BD11BC11BA83FF0BC086B3867041F065
:1009000080E48BBF80E385BF98BB78948895F8948A
:1009100080E285BF8BE080BD81E188BB89E087BB39
:1009200080E185BB80E48BBF82E083BF8BB78064AE
:100930008BBF8BE48093740088E081BD81E080935D
:10094000200178942DDF9091840019160CF025C1B8
:1009500080918100CCE0D0E0C81BD109C857DF4F9F
:100960009350809180008D3209F0E0C08AE5809339
:100970006100983009F007C19881892F807609F0CD
:1009800067C0109272008981882359F41092730015
:1009900082E790E0909383008093820090E822E0C9
:1009A000BEC0853021F48A8180938500ABC086303B
:1009B000C1F58B81813049F48EE190E09093830002
:1009C0008093820090EC22E1AAC0823049F480E357
:1009D00090E0909383008093820090EC22E29FC08D
:1009E000833021F4CE0157DE282F62C0813249F4D2
:1009F00082E490E0909383008093820090EC29E061
:100A00008EC0823249F482E590E090938300809317
:100A1000820090EC27E783C0CE013DDE282F90ECCA
:100A200074C0883019F487E890E05CC0893021F404
:100A30008A818093870066C08A3019F482E790E04B
:100A400051C08B3009F05EC08BE4809374005AC0B3
:100A50009076903209F056C08981823009F440C006
:100A6000833020F4813009F04DC006C0893091F107
:100A70008A3009F047C03DC08B818330D9F41A8198
:100A800010939E00042D812FC9DE173031F400230E
:100A900009F441108062C09B80619093A000809314
:100AA0009F008EE990E090938300809382002E81D6
:100AB00090E82BC080916800882319F401DF882317
:100AC00009F180E291E0909383008093820090E8A6
:100AD00025E025C087E093E09B838A8390E817C0D8
:100AE00088E690E0909383008093820090E821E074
:100AF00016C08B818093680081E090E090931F0185
:100B000080931E0190E820E00AC02F3F41F48881C5
:100B100087FD02C08FEF01C08E819F7738C08F8123
:100B20008823A1F58E81821790F130C080916500F5
:100B300087FD29C0923009F588818730F1F4198149
:100B40001F7C67DD86E050DD882339F4812F4CDD82
:100B5000882319F480E090E002C081E090E0482E04
:100B6000882319F40FE0202E2122898184FF02C0FE
:100B7000C09801C0C09A90E007C08EE180936100E8
:100B800090E08FEF04C090E880E001C0822F909346
:100B9000650080936000109284008091610084FF62
:100BA00049C0809160008F3F09F444C0182F8930FC
:100BB00008F018E0811B809360008091650080FD43
:100BC00002C00BE401C003EC8F5F809365002091AD
:100BD00082003091830086FD05C0D901912FEAE69D
:100BE000F0E011C0AAE6B0E080E090E006C0F901B4
:100BF000E80FF91FE491ED9301961817C1F705C0AE
:100C00008D91819391509923D9F7F901E10FF11D4D
:100C1000F0938300E09382008AE690E0612F6CDB22
:100C2000183019F08FEF80936000009369001C5F0B
:100C3000109361009AE086B3867031F49150D9F731
:100C40001092850010927F008E9B04C039DE8111C6
:100C50008F9A8E988091620084FF74CE8F9B72CEA3
:100C60008091620084FF0BC08091740098E889270E
:100C700080937400E0E2F1E0A5E7B0E006C08AE509
:100C800080936200F7CF81918D9381E0E532F80780
:100C9000D1F785E790E065E02FDB89E08093620083
:080CA0008F9850CEF894FFCFAD
:040CA800FF5A5A0095
:00000001FF
